:1000000019C032C031C030C02FC02EC02DC02CC08E
:100010002BC02AC029C028C027C026C025C024C0A4
:1000200023C022C021C020C01FC01EC01DC01CC0D4
:100030001BC01AC011241FBECFEFD2E0DEBFCDBF60
:1000400011E0A0E0B1E0EAE0F2E002C005900D921C
:10005000A030B107D9F711E0A0E0B1E001C01D92D6
:10006000A030B107E1F701C0CBCFCBEDD2E0DEBFCE
:10007000CDBFA3D0789480EF8BB98AB915B814B8E6
:10008000BB245B2CAB2CEE24FF243701470181E01D
:1000900090E00E2C02C0880F991F0A94E2F784B9F1
:1000A000CC24DD2484010E0D1F1D0C0D1D1D1E0111
:1000B0000894211C311C020D131D8C2D90D0F801C9
:1000C00080838B3038F5EC14FD0451F481E090E02E
:1000D0000E2C02C0880F991F0A94E2F7582A1AC002
:1000E00085E090E08C199D09E816F90651F481E04D
:1000F00090E00E2C02C0880F991F0A94E2F7B82AEC
:1001000009C081E090E00E2C02C0880F991F0A946C
:10011000E2F7A82AF301EE0DFF1DEC0DFD1DE20D27
:10012000F31D80818B50833F48F481E090E00E2CDA
:1001300002C0880F991F0A94E2F7A82A0894C11CEC
:10014000D11CF6E0CF16D1040CF4ACCF0894E11C1E
:10015000F11C85E090E0880E991E680E791E8E15C0
:100160009F050CF094CF8FEFEFE35E1631F4BB20C8
:1001700069F4AA2059F48FEE1EC0552039F4FFE32C
:10018000BF1621F4AA2011F48FED15C0A1108F7BAA
:100190009FE3591621F4BB2021F08F7B02C055202C
:1001A00021F0EFE3BE1609F48F7BFEE3F51518F09E
:1001B000FB1508F08F778BB963CF809164008E7F39
:1001C0008093640080E480937C0087E980937A00C8
:1001D00010927B008FE380937E000895089586300F
:1001E00018F080E090E00895805A80937C00809120
:1001F0007A00806480937A0080917A0086FDFCCF3B
:0A0200008091790099270895089570
:00000001FF
